:100000008A0103283A298312860185010630831666
:100010009F001F3085008601831205081039003CBF
:1000200003191A28050886000A30A10002208A1147
:100030000A1239298312A3010830831223020130E6
:1000400003180301003C0319662886012308A00059
:10005000003C031D2D2806145D2883122008013C56
:10006000031D342886145D2883122008023C031DDA
:100070003B2806155D2883122008033C031D4228F7
:1000800086155D2883122008043C031D49280616A6
:100090005D2883122008053C031D502886165D2824
:1000A00083122008063C031D572806175D2883127B
:1000B0002008073C031D5D288617FF308312A1002E
:1000C00002208A110A128312A30A1C2883128601B5
:1000D000A301083083122302013003180301003CFE
:1000E0000319B2282308A000003C031D7928061438
:1000F000A92883122008013C031D80288614A92802
:1001000083122008023C031D87280615A9288312A4
:100110002008033C031D8E288615A9288312200879
:10012000043C031D95280616A92883122008053CC7
:10013000031D9C288616A92883122008063C031D4F
:10014000A3280617A92883122008073C031DA92805
:100150008617FF308312A10002208A110A1283122F
:10016000A30A692883128601FF30A10002208A11A8
:100170000A123F3083128600FF30A10002208A114C
:100180000A12063083128600FF30A10002208A1175
:100190000A125B3083128600FF30A10002208A1110
:1001A0000A124F3083128600FF30A10002208A110C
:1001B0000A12663083128600FF30A10002208A11E5
:1001C0000A126D3083128600FF30A10002208A11CE
:1001D0000A127D3083128600FF30A10002208A11AE
:1001E0000A12073083128600FF30A10002208A1114
:1001F0000A127F3083128600FF30A10002208A118C
:100200000A126F3083128600FF30A10002208A118B
:100210000A12773083128600FF30A10002208A1173
:100220000A127C3083128600FF30A10002208A115E
:100230000A12393083128600FF30A10002208A1191
:100240000A125E3083128600FF30A10002208A115C
:100250000A12793083128600FF30A10002208A1131
:100260000A12713083128600FF30A10002208A1129
:100270000A120C2873308312A20000000000000054
:10028000000000000000000000000000000000006E
:0E029000A20B3E290000A10B3A290000080035
:00000001FF
